:020000020000FC
:02000000A8C096
:020008005DC0D9
:10000E0018C001020507446F75626C65466F782053
:10001E004D756C7469706C65786572532052657697
:10002E002E20312E30610D0000006572726F720D40
:10003E0000006FB6ACB15C9909C082FD13C081FFA0
:10004E0007C0AD3009F48D7F8A2E88606FBE18957B
:10005E008260A43221F08A2E88606FBE189584606B
:10006E006FBE18958B7FA43221F48A2E88606FBEE6
:10007E0018958D7FA03379F0A13389F0A23399F0D2
:10008E00A333A9F0AF3321F0A33711F06FBE18954B
:10009E00EA2E6FBE189532E041E06FBE189534E03F
:1000AE0048E06FBE189530E240E16FBE189530E81B
:1000BE0040E46FBE18956FB680FD03C083FD15C07A
:1000CE0020C06A95F1F4DD2011F48E7F1AC0DA9407
:1000DE005694A8B320F0A32BA8BB68E012C03095AD
:1000EE00A3233095A8BB68E00CC0877F8160582C95
:1000FE00509469E0D62E68E0A8B33095A3233095CE
:10010E00A8BBA6B3A42370FD13C0AA2361F018C028
:10011E00AA2319F47E7F942B13C07E7F81605D9B92
:10012E00FECF1CB80DC07160B9E09B2E2AE008C04E
:10013E00215031F49A9461F3A095AF5F179428E0A3
:10014E006FBE18950FED0DBF06EA07BB0FEF08BB8C
:10015E0008E90AB900E409B900270FBD09E00EBD90
:10016E0000270BBD01E80ABD00E409BF32E041E003
:10017E00EE248827772766249927DD24DA94FF2733
:10018E00DD277894EE2009F4FDCF0E2D0F3371F09C
:10019E000337C1F0E8E35D9901C0FDCFC895E39543
:1001AE00002D0CB90D30B9F7EE24ECCFE4E15D99DA
:1001BE0001C0FDCFC895E395002D0CB90D30B9F7F0
:1001CE00EE24E0CFD8E0C92F5D9901C0FDCFCC0F52
:1001DE0010F401E301C000E30CB9DA95A9F7EE249F
:0E01EE0099275D9901C0FDCF0DE00CB9CBCF74
:00000001FF
